:100000000C944E050C9495050C9495050C9495054F
:100010000C9495050C9495050C9495050C949505F8
:100020000C9495050C9495050C9495050C94640C12
:100030000C94130D0C94F31B0C9495050C949505DE
:100040000C9495050C9495050C9495050C94671CDF
:100050000C9495050C9495050C9495050C949505B8
:100060000C9495050C9495050C9495050C949505A8
:100070000C9495059206950698069B069E06A10689
:10008000A406800DA20D950EA20D950EE70D0A0E89
:10009000950E5F0E720E0B120B1235123512901266
:1000A000C412B414B414DB12B414C613C6138C14E3
:1000B000B414B414A1147E10360E0F12272D7F37FE
:1000C000383334132F2E7C7D29283130742A7879E7
:1000D00039042B14351E7B641D161A081F207A1B49
:1000E0000709151721222C06190A1C182324650557
:1000F000110B0D0C25260A002530325800626F7551
:100100006E6365213A20000A4B6579626F61726403
:100110002073746172742E0A000A55534220636F73
:100120006E666967757265642E0A000A0A544D4B43
:100130003A35386362626235632F4C5546410A0A8C
:10014000000E0341006C00700073003600340000A4
:1001500000080354004D004B00000004030904098B
:10016000027400040100A03209040000010301012F
:100170000009211101000122400007058103080048
:100180000A09040100010301020009211101000113
:10019000224D000705820308000A0904020001033A
:1001A0000000000921110100012236000705830328
:1001B00008000A09040300020300000009211101DC
:1001C0000001222200070584032000010705040323
:1001D0002000011201100100000008EDFE6464011E
:1001E00000010200010631FF0974A1010975150023
:1001F00026FF009520750881020976150026FF006C
:10020000952075089102C005010980A1018502169B
:1002100001002637001A81002AB700751095018168
:1002200000C0050C0901A1018503160100269C02EE
:100230001A01002A9C02751095018100C005010970
:1002400002A1010901A100050919012905150025CF
:10025000019505750181029501750381010501096B
:100260003009311581257F950275088106093815F9
:1002700081257F950175088106050C0A38021581D4
:10028000257F950175088106C0C005010906A101F9
:10029000050719E029E71500250195087501810278
:1002A0009501750881010508190129059505750154
:1002B00091029501750391010507190029FF1500A9
:1002C00026FF00950675088100C0636F6E73756D1B
:1002D00065723A20253034580A0073797374656D5D
:1002E0003A20253034580A000A00253032582000C0
:1002F0006B6579626F6172643A20004C45443A2024
:10030000253032580A00253032583A2025303862DC
:1003100025730A00722F632030313233343536377B
:100320000A00646F6E652E0A00626F6F746D6167FC
:100330006963207363616E3A202E2E2E2000290AF5
:10034000002575002F002575005D2800256400201C
:1003500000256400200025640020002564007C0046
:1003600025303258006D6F7573656B6579205B625F
:10037000746E7C782079207620685D287265702FF5
:1003800061636C293A205B006D6B5F776865656C13
:100390005F74696D655F746F5F6D6178203D2025C6
:1003A000640A006D6B5F776865656C5F6D61785F8F
:1003B0007370656564203D2025640A006D6B5F7471
:1003C000696D655F746F5F6D6178203D2025640AFB
:1003D000006D6B5F6D61785F7370656564203D20B3
:1003E00025640A006D6B5F696E74657276616C20BE
:1003F0003D2025640A006D6B5F64656C6179203D6A
:100400002025640A006D6B5F776865656C5F7469B1
:100410006D655F746F5F6D6178203D2025640A0013
:100420006D6B5F776865656C5F6D61785F73706534
:100430006564203D2025640A006D6B5F74696D65FD
:100440005F746F5F6D6178203D2025640A006D6BDD
:100450005F6D61785F7370656564203D2025640A77
:10046000006D6B5F696E74657276616C203D20254E
:10047000640A006D6B5F64656C6179203D202564C2
:100480000A000A00257500363A20776865656C5FBA
:1004900074696D655F746F5F6D61783A20000A0062
:1004A000257500353A20776865656C5F6D61785F0A
:1004B00073706565643A20000A00257500343A209F
:1004C00074696D655F746F5F6D61783A20000A0032
:1004D000257500333A206D61785F73706565643A05
:1004E00020000A00257500323A20696E7465727624
:1004F000616C286D73293A20000A00257500313A95
:100500002064656C6179282A31306D73293A2000A6
:100510000A092D2056616C756573202D0A004D3E29
:10052000004D25643E20003F0073657420646566BD
:1005300061756C740A00433E20007768657265201F
:1005400064656C74613A20637572736F723D2564E3
:100550002C20776865656C3D25640A5365652068C5
:100560007474703A2F2F656E2E77696B69706564AD
:1005700069612E6F72672F77696B692F4D6F757385
:10058000655F6B6579730A000A092D204D6F7573DD
:10059000656B6579202D0A4553432F713A097175B2
:1005A00069740A313A0964656C6179282A31306DC1
:1005B00073290A323A09696E74657276616C286D26
:1005C00073290A333A096D61785F73706565640A4F
:1005D000343A0974696D655F746F5F6D61780A35CF
:1005E0003A09776865656C5F6D61785F7370656502
:1005F000640A363A09776865656C5F74696D655F92
:10060000746F5F6D61780A0A703A097072696E746E
:100610002076616C7565730A643A097365742064A9
:10062000656661756C74730A75703A092B310A64DA
:100630006F776E3A092D310A706775703A092B3160
:10064000300A7067646F776E3A092D31300A0A7389
:1006500070656564203D2064656C7461202A206D9E
:1006600061785F7370656564202A20287265706503
:100670006174202F2074696D655F746F5F6D6178A0
:10068000290A003F004D3E2000433E20004C2564D7
:100690000A000A092D20436F6E736F6C65202D0AC6
:1006A0004553432F713A09717569740A6D3A096DA2
:1006B0006F7573656B65790A000A092D204D6167B6
:1006C0006963202D0A643A0964656275670A783A9D
:1006D000096465627567206D61747269780A6B3AA6
:1006E000096465627567206B6579626F6172640A7F
:1006F0006D3A096465627567206D6F7573650A767A
:100700003A0976657273696F6E0A733A0973746198
:100710007475730A633A09636F6E736F6C65206D4D
:100720006F64650A302D343A096C61796572302D39
:1007300034284631302D4634290A506175733A0900
:10074000626F6F746C6F616465720A653A09656502
:1007500070726F6D0A000A002575002E6E6B726F45
:100760003A20000A002575002E737761705F626180
:10077000636B736C6173685F6261636B73706163F9
:10078000653A20000A002575002E737761705F6757
:10079000726176655F6573633A20000A0025750013
:1007A0002E6E6F5F6775693A20000A002575002E6E
:1007B000737761705F72616C745F726775693A20FC
:1007C000000A002575002E737761705F6C616C7490
:1007D0005F6C6775693A20000A002575002E636119
:1007E00070736C6F636B5F746F5F636F6E74726F47
:1007F0006C3A20000A002575002E737761705F63E4
:100800006F6E74726F6C5F636170736C6F636B3A61
:1008100020000A0025303258006B65796D61705FE9
:10082000636F6E6669672E7261773A20000A002551
:1008300075002E6D6F7573653A20000A00257500EE
:100840002E6B6579626F6172643A20000A0025752B
:10085000002E6D61747269783A20000A00257500D7
:100860002E656E61626C653A20000A0025303258B0
:100870000064656275675F636F6E6669672E72619B
:10088000773A20000A0025750064656661756C740E
:100890005F6C617965723A20003F0074696D657222
:1008A0005F72656164333228293A202530346C58F0
:1008B0000A006B6579626F6172645F69646C653AA6
:1008C0002025580A006B6579626F6172645F7072EF
:1008D0006F746F636F6C3A2025580A00686F7374E9
:1008E0005F6B6579626F6172645F6C656473282900
:1008F0003A2025580A000A092D2053746174757333
:10090000202D0A004743433A20352E342E30204113
:1009100056522D4C4942433A20322E302E3020413F
:1009200056525F415243483A2061767233350A008D
:100930004F5054494F4E533A204C55464120424F58
:100940004F544D41474943204D4F5553454B455911
:100950002045585452414B455920434F4E534F4C1C
:100960004520434F4D4D414E44204B45594D41503C
:100970005F53454354494F4E20343039360A0042C4
:1009800055494C443A203538636262623563202809
:1009900031313A31303A3031204D617920333020D5
:1009A00032303139290A005649443A2030784645D8
:1009B000454428544D4B29205049443A203078363C
:1009C00034363428416C7073363429205645523AF7
:1009D000203078303030310A00444553433A2054B7
:1009E0004D4B206B6579626F617264206669726D30
:1009F0007761726520666F7220416C707336340ABD
:100A0000000A092D2056657273696F6E202D0A0049
:100A10000A6D6F7573653A206F66660A000A6D6F1E
:100A20007573653A206F6E0A000A6B6579626F61B3
:100A300072643A206F66660A000A6B6579626F61BC
:100A400072643A206F6E0A000A6D61747269783AB6
:100A5000206F66660A000A6D61747269783A206FC9
:100A60006E0A000A64656275673A206F6E0A000AB2
:100A700064656275673A206F66660A000A0A626FEB
:100A80006F746C6F616465722E2E2E2000433E20C1
:100A9000006565636F6E6669673A0A0011241FBEC0
:100AA000CFEFD4E0DEBFCDBF04B603FE27C08091F8
:100AB000110390911203A0911303B0911403873096
:100AC000904BA740B04BD1F4109211031092120337
:100AD000109213031092140314BE84B7877F84BF4F
:100AE0000FB6F894A89580916000886180936000AB
:100AF000109260000FBEE0E0F8E3099511E0A0E07D
:100B0000B1E0E4E5F0E502C005900D92A833B1072D
:100B1000D9F723E0A8E3B1E001C01D92A131B207EB
:100B2000E1F70E944D090C9428280C940000FF93D3
:100B3000EF93E0913801F0913901309709F0099570
:100B4000EF91FF910895FC018591803011F0EFDF66
:100B5000FBCF0895FF27E0E230E247FF0CC041954C
:100B600097FF09C0EDE26095709580959095611DA5
:100B7000711D811D911D27FF02C0219530E350E2B8
:100B8000AA27660F771F881F991FAA1FA41710F0A6
:100B9000A41B63955A95A9F7AA3008F0A95FA05D38
:100BA000AF93F395611571058105910541F7ED321C
:100BB00011F4EF93F395F21718F43F93F395FBCFED
:100BC0008F91B5DFFA95E1F70895E991F991859153
:100BD000803021F0853219F0AADFF9CF089520E0A6
:100BE000E89455915532C1F3503311F468945591FE
:100BF0005A3348F4505390F3220F022E220F220F43
:100C0000200D250FF4CF0EF421958991999153363B
:100C100019F3533729F1533559F1BC018827992726
:100C2000E8945C3621F489919991689455915436F1
:100C300039F446EF7EF077FF0DC08FEF9FEF0AC0CB
:100C400055374AE039F0583540E121F0523642E05C
:100C500009F00895FF93EF937DDFEF91FF91B7CFF8
:100C6000FF93EF93FC0181918030B9F360DFFBCFFC
:100C7000FF93EF9368DFF1CFDF93CF93CDB7DEB76C
:100C80002596A3DFCF91DF9108958AB180788AB944
:100C90008BB180788BB93A98429808950E944506A6
:100CA00084B114B885B18FEF85B9E2E4F1E0AAE32D
:100CB000B1E011921D9221E0EA34F207D1F7809160
:100CC000F20282608093F2023D9A459A8FEF99E694
:100CD00028E1815090402040E1F700C000003D989D
:100CE00045980895CF92DF92EF92FF920F931F9352
:100CF000CF93DF930AE311E0E801D12C85E0C82E01
:100D000098EFE92E90E0F92E8D2D90E0FC013197BF
:100D1000E730F10520F4E65CFF4F0C94DD27509A94
:100D2000589814C0519A599811C0529A5A980EC0A6
:100D3000539A5B980BC0549A5C9808C0559A5D987A
:100D400005C0569A5E9802C03A9A429880EA8A95FF
:100D5000F1F783B180959881981739F18883809154
:100D60000001882301F18091F20280FF04C08DEF21
:100D700090E00E94A3058091F20280FF0CC0809158
:100D800000011F928F93FF92EF920E943C060F90FA
:100D90000F900F900F908091F20280FF04C086EFB9
:100DA00090E00E94A305C09200010E944506D394E2
:100DB000219698E0D912A8CF809100018823B1F044
:100DC000815080930001882339F0AFE9BFE011978B
:100DD000F1F700C000000AC0E2E4F1E0D8018D9113
:100DE0008D018193B1E002341B07C1F781E0DF91EF
:100DF000CF911F910F91FF90EF90DF90CF900895CA
:100E0000E82FF0E0EE5BFE4F8081089581FF03C084
:100E10003D9A459A08953D984598089580915602C7
:100E20000895CF93DF9300D01F92CDB7DEB79C011A
:100E300080910703843019F593E099833B832A83DB
:100E40009093E9008FEF9091E800815095FD06C0E6
:100E500095ED9A95F1F700008111F5CF8091E800AA
:100E600085FF0DC040E050E063E070E0CE010196E8
:100E70000E94760A8091E8008E778093E8000F90B8
:100E80000F900F90DF91CF910895CF93DF9300D013
:100E90001F92CDB7DEB720910703243031F522E051
:100EA0002983805891099B838A8383E08093E9009A
:100EB0008FEF9091E800815095FD06C095ED9A95D1
:100EC000F1F700008111F5CF8091E80085FF0DC09A
:100ED00040E050E063E070E0CE0101960E94760AA7
:100EE0008091E8008E778093E8000F900F900F902C
:100EF000DF91CF910895209107032430F1F422E08F
:100F00002093E9002FEF3091E800215035FD06C015
:100F100035ED3A95F1F700002111F5CF2091E80069
:100F200025FF0BC040E050E065E070E00E94760ACB
:100F30008091E8008E778093E8000895CF93DF9347
:100F400020910703243049F521E02093E90021E8AE
:100F5000215059F03091E80035FD07C0EFE3F1E092
:100F60003197F1F700C00000F3CF2091E80025FF92
:100F700014C0EC0140E050E068E070E00E94760AA6
:100F80008091E8008E778093E80088E0FE01AEE46F
:100F9000B2E001900D928A95E1F7DF91CF9108952B
:100FA000CF93C0914C01C1110BC00E94311C643C15
:100FB00079408105910520F081E080934C01C1E0EA
:100FC0008C2FCF910895CF93C82F0E94D0078823EC
:100FD00009F448C00FB607FE45C08091070384306E
:100FE00009F040C08091E9008F702091EC00922FB1
:100FF000917020FD90E8892B94E09093E900909106
:10100000EB0090FF2CC09091EE0097FF28C09091CC
:10101000040120910301291709F447C02091E80039
:1010200025FF1DC0E0910101F0910201E90FF11DC2
:1010300030819F5F209105019223909304013093AA
:10104000F1009091E80095FDE2CF9091E80090FFCB
:10105000DECF9091E8009E779093E800D8CF8F7014
:101060008093E9008091030190E0AC014F5F5F4FF6
:1010700030910501232F30E02423352340910401D2
:1010800050E024173507D1F0209101013091020181
:10109000F901E80FF91FC083809103018F5F9091E0
:1010A000050189238093030109C09091E80095FF11
:1010B000D6CFC093F1008F708093E90080E0CF918C
:1010C00008950895089542E061EC81E00E947A0B52
:1010D00042E061EC82E00E947A0B42E061EC83E046
:1010E0000E947A0B42E261EC84E00C947A0B8091CE
:1010F0000903833009F453C030F4813071F0823039
:1011000009F48CC008958A3009F478C08B3009F452
:101110005EC0893009F09AC020C080910803813AEE
:1011200009F094C08091E800877F8093E800809167
:101130000C0390910D03892B21F468E08EE492E07A
:1011400003C060E080E090E070E00E94C10A8091FE
:10115000E8008B778093E80008958091080381323E
:1011600009F074C080910C0390910D03892B09F054
:101170006DC08091E800877F8093E8008091E8004F
:1011800082FD05C0809107038111F8CF5FC0809177
:10119000F100809356028091E8008B7753C08091D4
:1011A0000803813A09F052C080910C0390910D031D
:1011B000892B09F04BC08091E800877F8093E8007D
:1011C0008091E80080FFFCCF8091100136C08091B3
:1011D00008038132D9F580910C0390910D03892B7E
:1011E000A9F58091E800877F8093E8000E94AF0B0B
:1011F00080910A03809310010C94D4148091080309
:10120000813221F58091E800877F8093E8000E9479
:10121000AF0B80910B0380935702089580910803D0
:10122000813AA1F48091E800877F8093E800809163
:10123000E80080FFFCCF809157028093F1008091FD
:10124000E8008E778093E8000C94AF0B08958091AE
:10125000560280934D01109256020E9419100C9470
:10126000D4140C9427090E94B21B80910503882393
:1012700029F00E94DB1B81110C94600A08950E94E2
:10128000EF1B80914D018093560208950C943F0905
:1012900008950C9448090C944809CF9384B7877F2C
:1012A00084BF0FB6F894A895809160008861809300
:1012B0006000109260000FBE90E080E80FB6F894D6
:1012C00080936100909361000FBE83EE97E00E94CF
:1012D000841B86E091E00E94AD0E8BE291E00E94BB
:1012E000A3050E944B090E946C0F0E94010C0E94F2
:1012F000540C8091E20084608093E20078940E9414
:101300006E0F80910703843019F00E944809F9CFCD
:1013100089E191E00E94A3050E94490987E091E0DC
:101320000E94A305C4E080910703853019F40E9450
:101330003309F9CF0E94740F2091E4003091E50049
:1013400080914A0190914B012817390761F38091F0
:10135000E4009091E50090934B0180934A010E9434
:10136000D007882301F3809107038430E1F6809150
:10137000E9008F702091EC00922F917020FD90E891
:10138000892BC093E9009091EB0090FF3FC09091B2
:10139000EE0097FF3BC090910401209103012917B3
:1013A00009F12091E80025FF1DC0E0910101F091B5
:1013B0000201E90FF11D30819F5F20910501922309
:1013C000909304013093F1009091E80095FDE3CFF4
:1013D0009091E80090FFDFCF9091E8009E77909386
:1013E000E800D9CF9091F200992381F09091E80024
:1013F00090FF0CC09091E80095FF03C01092F1009F
:10140000F9CF9091E8009E779093E8008F708093D9
:10141000E90089CF292F332723303105C9F060F443
:101420002130310581F02230310509F041C084E7D7
:1014300090E02FE531E040C021323105E1F0223269
:10144000310531F135C082E190E023ED31E034C067
:1014500099278130910549F028F0029749F5E1E498
:10146000F1E005C0EBE5F1E002C0E1E5F1E08491D7
:1014700090E09F0121C06430D8F4E62FF0E0EE0F39
:10148000FF1FEB5DFE4F2081318189E090E014C0A9
:10149000643070F470E0FB01EE0FFF1FE35EFE4F5F
:1014A00020813181FB01E75EFE4F808190E004C026
:1014B00080E090E020E030E0FA013183208308955D
:1014C00084E089BD86E089BD09B400FEFDCF80912E
:1014D000D8008F7D8093D8008091E0008260809357
:1014E000E0008091E00081FDFCCF0895CF92DF9273
:1014F000EF92FF920F931F93CF93DF93EC018B0139
:101500007A010E94CE0B811133C0E114F10439F04D
:10151000F70180819181081B190BC80FD91FC12CBD
:10152000D12C0115110519F18091E80085FD16C037
:101530008091E8008E778093E800E114F10449F08F
:10154000F70180819181C80ED91ED182C08285E0C9
:101550000FC00E94CE0B882321F30AC0899180938B
:10156000F10001501109FFEFCF1ADF0ADACF80E056
:10157000DF91CF911F910F91FF90EF90DF90CF906F
:10158000089520910E0330910F032617370748F076
:101590006115710539F42091E8002E772093E80059
:1015A00001C0B901FC0120E06115710561F1809174
:1015B00007038823D9F18530D9F18091E80083FDB4
:1015C00039C08091E80082FD2BC08091E80080FF47
:1015D000EBCF8091F20090E06115710551F08830F9
:1015E000910538F421912093F10061507109019621
:1015F000F3CF21E0089709F020E08091E8008E7792
:101600008093E800D1CF2111D2CF0AC08091070387
:10161000882361F0853061F08091E80083FD0AC085
:101620008091E80082FFF2CF80E0089582E0089583
:1016300083E0089581E0089520910E0330910F0317
:101640002617370748F06115710539F42091E80035
:101650002E772093E80001C0B901FC0120E061155C
:10166000710579F180910703882309F43DC0853025
:1016700009F43CC08091E80083FD3AC08091E80005
:1016800082FD2CC08091E80080FFE9CF8091F200BC
:1016900090E06115710559F08830910540F424916E
:1016A0002093F1003196615071090196F2CF21E04B
:1016B000089709F020E08091E8008E778093E80099
:1016C000CECF2111CFCF0AC080910703882361F0CC
:1016D000853061F08091E80083FD0AC08091E800C8
:1016E00082FFF2CF80E0089582E0089583E00895BC
:1016F00081E00895982F953068F59093E900981748
:1017000039F07091EC002091ED005091F00003C091
:10171000242F762F50E021FD02C09F5FECCF309147
:10172000EB003E7F3093EB003091ED003D7F309336
:10173000ED003091EB0031603093EB007093EC00E2
:101740002093ED005093F0002091EE0027FDE5CFAF
:1017500080E008958F708093E90081E00895809182
:10176000080387FF11C08091E80082FD05C08091C9
:1017700007038111F8CF11C08091E8008B770BC06F
:1017800080910703882349F08091E80080FFF8CF1B
:101790008091E8008E778093E80008952091E4001E
:1017A0003091E50095E64091EC00842F817040FF78
:1017B00023C08091E80080FD1DC08091070388232D
:1017C00099F0853099F08091EB0085FD11C0409132
:1017D000E4005091E5002417350729F3915011F0EA
:1017E0009A01E1CF84E0089582E0089583E00895AE
:1017F00081E0089580E008954091E80042FFDDCF48
:1018000008950E945E0C0E94610CE0EEF0E0808181
:1018100081608083E8EDF0E080818F77808319BC60
:10182000E3E6F0E0808181608083109206030895F2
:101830000E945E0C0E94610C8091D8008F7780938B
:10184000D8008091D80080688093D8008091D8001B
:101850008F7D8093D80084E089BD86E089BD09B47E
:1018600000FEFDCF109207031092030310920503B0
:101870001092040342E060E080E00E947A0B8091C5
:10188000E1008E7F8093E1008091E200816080938F
:10189000E2008091E20088608093E2008091E000A5
:1018A0008E7F8093E0000895E3E6F0E080818E7FF4
:1018B000808381E0809306030C94180C1092E20060
:1018C00008951092E10008951F920F920FB60F92A3
:1018D00011242F933F934F935F936F937F938F9335
:1018E0009F93AF93BF93EF93FF938091E10082FFAB
:1018F0000BC08091E20082FF07C08091E1008B7FE6
:101900008093E1000E9462088091E10080FF19C08D
:101910008091E20080FF15C08091E2008E7F80936D
:10192000E2008091E20080618093E2008091D80023
:1019300080628093D80019BC85E0809307030E94E1
:1019400031098091E10084FF30C08091E20084FF82
:101950002CC084E089BD86E089BD09B400FEFDCFBE
:101960008091D8008F7D8093D8008091E1008F7E98
:101970008093E1008091E2008F7E8093E20080916D
:10198000E20081608093E20080910303882311F0DC
:1019900084E007C08091E30087FD02C081E001C0C0
:1019A00083E0809307030E9446098091E10083FF52
:1019B00029C08091E20083FF25C08091E100877FEC
:1019C0008093E10082E080930703109203038091EB
:1019D000E1008E7F8093E1008091E2008E7F809312
:1019E000E2008091E20080618093E20042E060E0EA
:1019F00080E00E947A0B8091F00088608093F00074
:101A00000E946108FF91EF91BF91AF919F918F91DB
:101A10007F916F915F914F913F912F910F900FBEEA
:101A20000F901F9018951F920F920FB60F921124CE
:101A30002F933F934F935F936F937F938F939F93D6
:101A4000AF93BF93CF93DF93EF93FF93C091E900E0
:101A5000CF708091EC00D82FD17080FDD0E810922B
:101A6000E9008091F000877F8093F00078940E94D5
:101A7000570D1092E9008091F00088608093F0008B
:101A8000CD2BCF70C093E900FF91EF91DF91CF9103
:101A9000BF91AF919F918F917F916F915F914F9186
:101AA0003F912F910F900FBE0F901F9018951F938D
:101AB000CF93DF93CDB7DEB7AA970FB6F894DEBF0A
:101AC0000FBECDBFE8E0F3E08091F100819323E009
:101AD000E031F207C9F70E9477088091E80083FFA0
:101AE00024C18091080390910903492F50E04A30A6
:101AF000510508F01AC1FA01EF5BFF4F0C94DD2786
:101B0000803881F0823809F010C180910C038F7009
:101B10008093E9008091EB0085FB882780F9109283
:101B2000E90006C080910403909105039111826041
:101B30009091E800977F9093E8008093F1001092D5
:101B4000F100C8C0282F2D7F09F0EFC0882319F0BD
:101B5000823061F0EAC080910A03813009F0E5C06B
:101B6000933009F080E0809305032BC080910A0335
:101B7000811127C080910C038F7009F4D6C0809327
:101B8000E9002091EB0020FF1CC0933021F48091EC
:101B9000EB00806214C09091EB0090619093EB0099
:101BA00021E030E0A90102C0440F551F8A95E2F7F9
:101BB0004093EA001092EA008091EB0088608093E5
:101BC000EB001092E9008091E800877F86C08111C8
:101BD000ACC010910A031F778091E3008078812BBD
:101BE0008093E3008091E800877F8093E8000E9463
:101BF000AF0B8091E80080FFFCCF8091E30080680C
:101C00008093E300111102C082E001C083E0809361
:101C100007038BC08058823008F087C080910A0388
:101C200090910B038C3D53E0950779F583E08A830F
:101C30008AE289834FB7F894DE01139620E03EE0F4
:101C400051E2E32FF0E050935700E49120FF03C0EE
:101C5000E295EF703F5FEF708E2F90E0EA3010F06A
:101C6000C79601C0C0968D939D932F5F243149F78D
:101C70004FBF8091E800877F8093E8006AE270E0C0
:101C8000CE0101960E94C10A14C0AE014F5F5F4FA2
:101C900060910C030E940A0ABC01892B09F445C01B
:101CA0009091E800977F9093E80089819A810E9443
:101CB0001C0B8091E8008B778093E80036C0803859
:101CC000A1F58091E800877F8093E800809103036D
:101CD0008093F1008091E8008E778093E8000E9465
:101CE000AF0B23C0811121C080910A0390910B0397
:101CF00099270297D4F48091E800877F8093E800C9
:101D000080910A03809303030E94AF0B8091030329
:101D1000811106C08091E30087FD02C081E001C00F
:101D200084E0809307030E9463088091E80083FFAA
:101D30000AC08091E800877F8093E8008091EB00E3
:101D400080628093EB00AA960FB6F894DEBF0FBEB8
:101D5000CDBFDF91CF911F91089590935D02809345
:101D60005C020895E0915C02F0915D02309721F0F1
:101D70000190F081E02D099480E00895EF92FF92A8
:101D80000F931F93CF93DF93E0915C02F0915D027C
:101D90003097B1F18C010280F381E02D099580919B
:101DA000F20282FF2DC080FF04C080EF92E00E940B
:101DB000A305E80118E08AEEE82E82E0F82E809173
:101DC000F20280FF0BC088811F928F93FF92EF92E7
:101DD0000E943C060F900F900F900F90115021968B
:101DE0001111EDCF8091F20280FF0AC088EE92E0DF
:101DF000DF91CF911F910F91FF90EF900C94A3056D
:101E0000DF91CF911F910F91FF90EF900895E09196
:101E10005C02F0915D02309721F00480F581E02DA5
:101E200009940895CF93DF9320915A0230915B0279
:101E30002817390709F190935B0280935A02E091C9
:101E40005C02F0915D023097B9F0EC010680F781F9
:101E5000E02D09958091F20282FF0EC080FF0CC038
:101E6000DF93CF938AED92E09F938F930E943C067D
:101E70000F900F900F900F90DF91CF910895CF9317
:101E8000DF9320915802309159022817390709F140
:101E90009093590280935802E0915C02F0915D02A8
:101EA0003097B9F0EC010084F185E02D099580911F
:101EB000F20282FF0EC080FF0CC0DF93CF938AEC4A
:101EC00092E09F938F930E943C060F900F900F908B
:101ED0000F90DF91CF9108950C941A100E941C1C52
:101EE0000E944E060C94431DBF92CF92DF92EF9258
:101EF000FF920F931F93CF93DF9300D000D01F92D8
:101F0000CDB7DEB70E9472060FE512E0F12C8F2DDF
:101F10000E940007B82EF801C080C82639F4F39457
:101F20000F5F1F4FF8E0FF12F2CF30C08091F20236
:101F300081FD0E941B10D12CEE24E3948C2D8E2168
:101F4000F9F0D982FA8291E08B2D8E2109F490E08C
:101F50009B830E94251C8160782F9D838C834981FF
:101F60005A816B818D810E94511049815A816B8108
:101F70007C818D810E949C1BF80180818E2580834D
:101F8000D394EE0CF8E0DF12D9CFC9CF8FEF89835D
:101F90008A831B820E94251C8160782F9D838C83FD
:101FA00049815A816B818D810E9451100E949B1B37
:101FB0000E94CA200E94B20E90915E02891741F1E0
:101FC0000E94B20E80935E029091F20292FF0EC0C8
:101FD00090FF0CC01F928F938BEF92E09F938F9393
:101FE0000E943C060F900F900F900F9080915E0220
:101FF0000F900F900F900F900F90DF91CF911F9146
:102000000F91FF90EF90DF90CF90BF900C94AD1B9D
:102010000F900F900F900F900F90DF91CF911F9125
:102020000F91FF90EF90DF90CF90BF9008950C94A8
:10203000060708950895EF92FF920F931F93CF9391
:10204000DF9384E193E00E94A305C0E0D0E08DE23D
:10205000E82E81E0F82E06E013E08C2F0E940007A6
:102060000E94891BFF92EF921F928F93DF93CF9371
:102070001F930F930E943C0621968DB79EB708963A
:102080000FB6F8949EBF0FBE8DBFC830D10529F79B
:10209000DF91CF911F910F91FF90EF9008950895D8
:1020A0000895CF93DF93CDB7DEB72B970FB6F89493
:1020B000DEBF0FBECDBF942F4F83252F5887698772
:1020C0007A878B874A855B85452B31F02F3F31F42A
:1020D00081E09F3F19F403C081E001C080E080FDF2
:1020E00007C04F81588569857A858B850E949C1B26
:1020F000DE01119686E0FD0111928A95E9F785E0EF
:10210000FE01379601900D928A95E1F749815A8137
:102110006B817C818D819E810E94F2172B960FB678
:10212000F894DEBF0FBECDBFDF91CF910895CF935E
:10213000882309F4A9C0C82F8238A1F40E94B20EE6
:1021400081FDA2C089E30E94E61A0E945E1B2FEF68
:1021500081EE94E0215080409040E1F700C0000003
:1021600089E315C08338C1F40E94B20E80FD8CC093
:1021700083E50E94E61A0E945E1B2FEF81EE94E039
:10218000215080409040E1F700C0000083E50E94AC
:10219000031BCF910C945E1B8438A1F40E94B20EF5
:1021A00082FD72C087E40E94E61A0E945E1B2FEF38
:1021B00081EE94E0215080409040E1F700C00000A3
:1021C00087E4E5CF8CEF8C0F813A20F080E58C0F0F
:1021D0008E3248F48C2F0E942A25811155C08C2FF5
:1021E0000E94E61AD6CF80E28C0F883048F4C77080
:1021F00081E001C0880FCA95EAF70E94241BC9CF6D
:102200008BE58C0F833078F4C53A29F0C63A31F06B
:1022100083E890E005C081E890E002C082E890E0A9
:10222000CF910C94120F88E58C0F853168F5C83A70
:1022300089F0C93A91F0CA3A99F0CB3AA1F0CC3A78
:10224000A9F0CD3AB1F0CE3AB9F0CF3AC1F080E082
:1022500090E017C082EE90E014C089EE90E011C0CB
:102260008AEE90E00EC085EB90E00BC086EB90E02C
:1022700008C083EB90E005C084EB90E002C087EBE0
:1022800090E0CF910C943F0FCF910895882309F4EB
:102290006AC08238A1F40E94B20E81FF64C089E353
:1022A0000E94E61A0E945E1B2FEF81EE94E02150FF
:1022B00080409040E1F700C0000089E315C08338FA
:1022C000B9F40E94B20E80FF4EC083E50E94E61A68
:1022D0000E945E1B2FEF81EE94E0215080409040E1
:1022E000E1F700C0000083E50E94031B0C945E1B15
:1022F0008438A1F40E94B20E82FF35C087E40E94A8
:10230000E61A0E945E1B2FEF81EE94E02150804080
:102310009040E1F700C0000087E4E6CF9CEF980F03
:10232000913A10F390E5980F9E32F0F290E2980FF8
:10233000983050F4877091E001C0990F8A95EAF7C0
:10234000892F0E942A1BD2CF9BE5980F933020F44F
:1023500080E090E00C94120F885A853120F480E0E0
:1023600090E00C943F0F0895882321F00E94241BD5
:102370000C945E1B0895882321F00E942A1B0C9464
:102380005E1B0895CF92DF92EF92FF920F931F93FF
:10239000CF93DF9300D000D01F92CDB7DEB76C0192
:1023A0000E94B01B8111E0C285E0F601DE011196AA
:1023B00001900D928A95E1F7F601408151812381C8
:1023C00034812115310531F05F3F31F481E04F3F19
:1023D00019F403C081E001C080E080FDC5C2F601B0
:1023E000F280E580E2948FE0E822722F3D832C8317
:1023F0006F2D8D810E945B1A8C010E945A1A0E94D7
:102400004A19E12FE295EF708E2F90E0FC01E55B19
:10241000FF4F0C94DD27812F807F1F70882311F0E0
:102420001295107FFF2049F0112309F452C2812F29
:102430000E94371B0E945E1B4CC2802F0E944611D7
:10244000112309F491C2812F0E943D1B0F900F9020
:102450000F900F900F90DF91CF911F910F91FF90F0
:10246000EF90DF90CF900C945E1B812F807F1F70C8
:10247000803211F01295107F002319F0013009F11C
:102480002BC0FF20A9F0EE2059F1F1E0812FEF12CF
:1024900028C00F900F900F900F900F90DF91CF9169
:1024A0001F910F91FF90EF90DF90CF900C94471BFE
:1024B000EE2021F081E0E81609F456C20E944A1B82
:1024C0002DC0FF20E9F0E5E0EE1508F44DC20E94B2
:1024D000211B812329F022C0FF20F1F0E11015C05B
:1024E000812F0F900F900F900F900F90DF91CF9151
:1024F0001F910F91FF90EF90DF90CF900C94B4114B
:10250000F4E0FE1508F430C209C0F601858180FFB1
:10251000E0C18F708583E4CFE110EEC1812F61C1EE
:10252000812F86958695837019F08130B9F01CC291
:10253000FF2019F0C801937002C080E090E00F9076
:102540000F900F900F900F90DF91CF911F910F91EF
:10255000FF90EF90DF90CF900C94120FFF2019F0B6
:10256000C801937002C080E090E00F900F900F9030
:102570000F900F90DF91CF911F910F91FF90EF90EF
:10258000DF90CF900C943F0F802FFF2019F00E9416
:10259000501F02C00E94B81F0F900F900F900F9015
:1025A0000F90DF91CF911F910F91FF90EF90DF90EF
:1025B000CF900C943D20812F837009F070C0F110F2
:1025C000D3C1202F229526952770220F220F602F2E
:1025D0006F70862F90E0A0E0B0E06C017D01022ECC
:1025E00004C0CC0CDD1CEE1CFF1C0A94D2F704FFC7
:1025F00012C08FE090E0A0E0B0E004C0880F991F07
:10260000AA1FBB1F2A95D2F7BC01CD01609570951A
:102610008095909503C060E070E0CB01169516950B
:1026200013701230B1F040F56C297D298E299F2955
:10263000113031F10F900F900F900F900F90DF91AC
:10264000CF911F910F91FF90EF90DF90CF900C945E
:102650006F196C297D298E299F290F900F900F905B
:102660000F900F90DF91CF911F910F91FF90EF90FE
:10267000DF90CF900C9489190E946F19C701B601A1
:102680000F900F900F900F900F90DF91CF911F91AF
:102690000F91FF90EF90DF90CF900C945519FF2091
:1026A00019F0812F817001C08695882309F45CC1DF
:1026B000202F229526952770220F220F602F6F70F2
:1026C000862F90E0A0E0B0E06C017D01022E04C0F6
:1026D000CC0CDD1CEE1CFF1C0A94D2F704FF12C0C8
:1026E0008FE090E0A0E0B0E004C0880F991FAA1F1F
:1026F000BB1F2A95D2F7BC01CD01609570958095DE
:10270000909503C060E070E0CB01169516951370AC
:102710001230B1F040F56C297D298E299F291130A6
:1027200031F10F900F900F900F900F90DF91CF919C
:102730001F910F91FF90EF90DF90CF900C94361A7D
:102740006C297D298E299F290F900F900F900F9053
:102750000F90DF91CF911F910F91FF90EF90DF903D
:10276000CF900C94481A0E94361AC701B6010F90F8
:102770000F900F900F900F90DF91CF911F910F91BD
:10278000FF90EF90DF90CF900C94241A003FC1F19E
:1027900028F480E4800F803250F096C0023F09F4A4
:1027A0005EC008F449C0033F09F46CC08DC0F02F2F
:1027B000F071EF2E812F8F71FF2051F00E94BD1913
:1027C000802FEE2019F08295807F8BCE8F7089CE7E
:1027D0000E94DE19802FEE2019F08295807F01C0C3
:1027E0008F700F900F900F900F900F90DF91CF91FF
:1027F0001F910F91FF90EF90DF90CF900C94BB1141
:10280000FF20A9F084E08E1508F4AEC0812F8F71EF
:102810000F900F900F900F900F90DF91CF911F911D
:102820000F91FF90EF90DF90CF900C94031AE5E0AA
:10283000EE1508F499C0EACFFF2099F0812F8F712F
:102840000F900F900F900F900F90DF91CF911F91ED
:102850000F91FF90EF90DF90CF900C94BD19FF2067
:1028600069F3812F8F710F900F900F900F900F9041
:10287000DF91CF911F910F91FF90EF90DF90CF905C
:102880000C94DE19FF2089F0812F8F710F900F902B
:102890000F900F900F90DF91CF911F910F91FF90AC
:1028A000EF90DF90CF900C94A8190F900F900F909D
:1028B0000F900F90DF91CF911F910F91FF90EF90AC
:1028C000DF90CF900C94A319FF2099F0EE2009F42B
:1028D000B5CF802F0F900F900F900F900F90DF913A
:1028E000CF911F910F91FF90EF90DF90CF900C94BC
:1028F0009710EE2009F4B5CF802F0F900F900F9016
:102900000F900F90DF91CF911F910F91FF90EF905B
:10291000DF90CF900C944611412F4F70602FC6016D
:102920000E94EE1C0F900F900F900F900F90DF9170
:10293000CF911F910F91FF90EF90DF90CF900C946B
:10294000A518412F4F70602FC6010F900F900F9068
:102950000F900F90DF91CF911F910F91FF90EF900B
:10296000DF90CF900C94F11C0F900F900F900F9070
:102970000F90DF91CF911F910F91FF90EF90DF901B
:10298000CF9008950E94441B0E94131B0E945E1B5F
:102990000E9470210E943D2080E090E00E94120F72
:1029A00080E090E00C943F0F0E94341B0C94C21402
:1029B0001F93CF93DF9300D000D01F92CDB7DEB727
:1029C000942F4983252F5A836B837C838D834C817D
:1029D0005D81452B31F02F3F31F481E09F3F19F4A9
:1029E00003C081E001C080E0182F117080FD31C06C
:1029F00049815A816B817C818D810E945B1A292FCC
:102A000022952F702C3030F42A30A0F4225022303E
:102A100030F022C02C30C9F02F30B9F01DC0853AFB
:102A200028F48430C0F4823028F415C090E2980F66
:102A3000983088F0883E30F4803E68F48450813AC3
:102A400058F409C0803F41F406C093FB112710F9E8
:102A500003C010E001C011E0812F0F900F900F9084
:102A60000F900F90DF91CF911F910895CF93DF9337
:102A700000D000D01F92CDB7DEB70F900F900F900F
:102A80000F900F90DF91CF910895CF93DF9300D0F7
:102A900000D000D0CDB7DEB726960FB6F894DEBFD3
:102AA0000FBECDBFDF91CF910895CF93DF93C0913B
:102AB000670280916802C817A1F0D0E0CE0166E0FD
:102AC00070E00E94B827FC01E759FD4F4081518119
:102AD00062817381848195810E9445152196C7701A
:102AE000E8CFDF91CF9108954091990250919A02D9
:102AF00060919B0270919C0280919D0290919E0238
:102B00000C9445151F93CF93DF9380919E0282957D
:102B10008F7009F066C080919B02882309F461C020
:102B20002091670210916802C0919902D0919A0297
:102B3000E0919C02F0919D0281E0CF3F09F080E09E
:102B4000482F211709F44DC0309721F0DF3F21F0C5
:102B500080E003C081E001C0842F30E080FD3DC0F3
:102B6000C90166E070E00E94B827DC01A759BD4F9B
:102B700011968C9111978D1330C08C918C132DC0B0
:102B800012968C911297811128C013968D919C9169
:102B900014978E179F0708F401978E1B9F0B883C94
:102BA0009105D8F480919E028F70806180939E027F
:102BB000C90166E070E00E94B827FC01E259FD4FB0
:102BC00090819F709061908389E992E00E94C21188
:102BD000DF91CF911F910C9455152F5F3F4F2770B8
:102BE000B0CFDF91CF911F910895AF92BF92CF9256
:102BF000DF92EF92FF920F931F93CF93DF93CDB7A6
:102C0000DEB761970FB6F894DEBF0FBECDBF7C0173
:102C100085E0F701DE011D9601900D928A95E1F79E
:102C2000D7014C9111962C9111971296DC90129726
:102C300013960D911C9114975091990260919A02EC
:102C400080919C0290919D02009731F06F3F31F48A
:102C500031E05F3F19F403C031E001C030E0B32F31
:102C6000B170BB2E30FD76C1A0909B02AA2009F462
:102C7000D2C030919E020817190728F0F801E81B0E
:102C8000F90BCF0104C080959095800F911FCC2443
:102C9000C394883C910588F0C12C307F09F0A6C010
:102CA000702F198B088B522F6D2D89890E94361534
:102CB00089E992E00E94C211C3C0832F807F09F08E
:102CC00059C0261315C0451313C0CD2CD11010C008
:102CD0003F70306130939E020E94741589E992E042
:102CE0000E94C21180919E02D70115968C9368C1F3
:102CF0000115110531F02F3F31F481E04F3F19F4F8
:102D000003C081E001C080E080FD03C081E08D252B
:102D100002C080E090E0B82FB170CB2E80FF1FC0C2
:102D2000E091670230916802E31709F425C1F0E0F1
:102D3000CF0166E070E00E94B827DC01A759BD4FC3
:102D400011968C911197281307C08C91481304C0D9
:102D500012968C91D81203C03196E770E5CFCD2C36
:102D6000DD2009F42DC180919E02816080939E0236
:102D7000C12C26C1261308C0451306C0D11004C0BB
:102D800080919E02D701B9C04D872E87DF86702FB4
:102D9000198B088B522F6D2D89890E94D814882396
:102DA000A1F1DD2091F120919E02822F82958F70FA
:102DB00090E0029774F08091990290919A0298871E
:102DC0008F8319861B870A872C87CE0107960E945E
:102DD000C21186E0F701A9E9B2E001900D928A954F
:102DE000E1F70E9482150E94741512C0261791F116
:102DF0004D872E87DF86702F198B088B522F6D2DF4
:102E000089890E94D814811139C0C7010E94C2115A
:102E1000CC24C394D5C00817190708F447C0F8019B
:102E2000E81BF90BCF01883C910508F444C0C12C84
:102E3000702F198B088B522F6D2D89890E943615A2
:102E4000E9E9F2E086E0DF011D928A95E9F70E9448
:102E50007415B6C04513CCCFD110CACF80919E0255
:102E6000F7018583C7010E94C21186E0E9E9F2E01B
:102E7000DF011D928A95E9F7CA2CA2C0DD2029F254
:102E800020919E02822F82958F7090E002970CF421
:102E9000A0CF8091990290919A029A8389831B8294
:102EA0001D830C832E83CE01019691CF8095909542
:102EB000800F911FB8CFCD2CDD2009F4A6CF2613AB
:102EC00033C0451331C020919E0220FD24C0822FC3
:102ED00082958F70482F50E041155105E1F0D701E0
:102EE00015962C9315974F30510549F08F5F982F09
:102EF0009295907F822F8F70892B15968C93C701A6
:102F00000E94C21186E0F701A9E9B2E001900D929A
:102F10008A95E1F79CCF86E0F701A9E9B2E001903C
:102F20000D928A95E1F74CC04D872E87DF86702F72
:102F3000198B088B522F6D2D89890E94D81481110D
:102F400048CF80919E02816080939E02C7010E94BB
:102F5000C21136C0DD2009F458CF4D872E87DF8699
:102F6000702F198B088B522F6D2D89890E94D814D0
:102F7000882309F44ACF2DCF702F198B088B522F3D
:102F80006D2D89890E945B1A292F22952F7022307E
:102F900028F49F7039F0811105C00BC0243028F44B
:102FA0009F7049F4805E883020F0C7010E94C211F2
:102FB000BC2CCB2C05C0F7019581907F99F7F9CFF8
:102FC0008C2D61960FB6F894DEBF0FBECDBFDF919A
:102FD000CF911F910F91FF90EF90DF90CF90BF9016
:102FE000AF900895CF93DF93CDB7DEB72C970FB690
:102FF000F894DEBF0FBECDBF4F83588769877A87AD
:103000008B879C87CE0107960E94F5158823D1F007
:103010009F8188852A853B85232B31F08F3F31F4B2
:1030200081E09F3F19F403C081E001C080E080FD92
:103030006FC04F81588569857A858B859C850E94F4
:10304000451566C086E0FE013796DE0111960190B7
:103050000D928A95E1F7FF81E8856A857B85611588
:10306000710531F0EF3F31F481E0FF3F19F403C007
:1030700081E001C080E080FD4BC08091680290E05B
:103080009C012F5F3F4F277033274091670250E02C
:103090002417350709F443C0F983EA837D836C83E1
:1030A00066E070E00E94B827DC01A759BD4F96E0AA
:1030B000FE01319601900D929A95E1F720936802F6
:1030C0000E94551525C090E066E070E00E94B82788
:1030D00087599D4F0E94F515882371F180916702F1
:1030E00090E066E070E00E94B827FC01E759FD4FD0
:1030F0004081518162817381848195810E9445154F
:103100008091670290E0019687709927809367020B
:1031100080916702909168028913D5CF0DC00E94FB
:10312000D4141092680210926702E9E9F2E086E096
:10313000DF011D928A95E9F72C960FB6F894DEBF51
:103140000FBECDBFDF91CF910895DF92EF92FF9236
:103150000F931F93CF93DF93FC01892B09F488C051
:10316000E12CF12CDD24D394EF0121968491853755
:1031700009F460C058F4843708F04EC0843008F079
:1031800068C08130D1F0823071F172C0883709F4A3
:103190005BC050F4863709F453C0873709F068C024
:1031A0008E2D0E94311B52C09CE7980F903708F07B
:1031B0005FC08F770E9446114EC08F010E5F1F4F78
:1031C000FE01849190E2980F983050F48770FD2DA5
:1031D00001C0FF0F8A95EAF78F2F0E94371B15C099
:1031E0000E94971014C08F010E5F1F4FFE01849143
:1031F00090E2980F983068F48770FD2D01C0FF0FA2
:103200008A95EAF78F2F0E943D1B0E945E1BE80102
:1032100022C00E944611FBCFCF010296FE01C4914D
:10322000CC2361F0EFE9FFE03197F1F700C0000037
:10323000C150F6CFCF010296FE01F490EC010BC015
:103240000E94211BE82E07C00E94341B0E945E1BB7
:1032500002C00E9497108F2D882341F0EFE9FFE014
:103260003197F1F700C000008150F6CFFE017CCF0E
:10327000DF91CF911F910F91FF90EF90DF90089514
:103280006093DF027093E0028093E1029093E20288
:103290000C94AC1B08956093E3027093E402809356
:1032A000E5029093E6020C94AB1B0F931F930091E1
:1032B000E3021091E4022091E5023091E602602BD6
:1032C000712B822B932B6093E3027093E402809323
:1032D000E5029093E6021F910F910C94AB1B0F93A4
:1032E0001F930091E3021091E4022091E5023091D6
:1032F000E60260237123822393236093E302709399
:10330000E4028093E5029093E6021F910F910C94E2
:10331000AB1B0F931F930091E3021091E4022091E5
:10332000E5023091E6026027712782279327609398
:10333000E3027093E4028093E5029093E6021F910A
:103340000F910C94AB1B60E070E0CB010C94401922
:103350000F931F9341E050E060E070E08A019B0111
:1033600004C0000F111F221F331F8A95D2F7C90115
:10337000B8011F910F910C9440190F931F9341E0D6
:1033800050E060E070E004C0440F551F661F771FD7
:103390008A95D2F78091DF029091E002A091E1023C
:1033A000B091E2028A019B01082B192B2A2B3B2B9F
:1033B000C901B8011F910F910C9440190F931F93ED
:1033C00041E050E060E070E004C0440F551F661F0C
:1033D000771F8A95D2F740955095609570958091AA
:1033E000DF029091E002A091E102B091E2028A0135
:1033F0009B01082319232A233B23C901B8011F91EC
:103400000F910C9440190F931F9341E050E060E03E
:1034100070E004C0440F551F661F771F8A95D2F7CE
:103420008091DF029091E002A091E102B091E2026E
:103430008A019B01082719272A273B27C901B801C0
:103440001F910F910C9440190F931F930091DF026D
:103450001091E0022091E1023091E202602B712B89
:10346000822B932B1F910F910C9440190F931F9354
:103470000091DF021091E0022091E1023091E2021E
:1034800060237123822393231F910F910C94401981
:103490000F931F930091DF021091E0022091E1024F
:1034A0003091E20260277127822793271F910F91A5
:1034B0000C94401908958F929F92AF92BF92DF9221
:1034C000EF92FF920F931F93CF93DF9300D000D022
:1034D0001F92CDB7DEB76B837C838D838A018C818D
:1034E0009D81892B31F01F3F31F481E04F3F19F46A
:1034F00003C081E001C080E080FF03C080E090E075
:1035000054C08B81882309F43DC08090DF029090E5
:10351000E002A090E102B090E2028091E30290917B
:10352000E402A091E502B091E602882A992AAA2A2B
:10353000BB2A2FE1E22EF12CD501C4010E2C04C0D0
:10354000B695A795979587950A94D2F780FD06C002
:1035500081E0E81AF10880F7D12C07C0DE2CB80111
:103560008E2D0E94BF1C019799F3E12FF0E093E0AC
:10357000EE0FFF1F9A95E1F7E156FD4FE00FF11DA9
:10358000D0820CC0E12FF0E083E0EE0FFF1F8A95A0
:10359000E1F7E156FD4FE00FF11DD08009831A835A
:1035A00069817A818D2D0E94BF1C0F900F900F9022
:1035B0000F900F90DF91CF911F910F91FF90EF909F
:1035C000DF90BF90AF909F908F9008952091110150
:1035D00030911201F90132969FEF40E05191851729
:1035E00089F09F3F19F4511101C0942F4F5F46306D
:1035F000A9F79F3F39F0F901E90FF11D97FDFA9501
:10360000828308950895E0911101F09112019F01C4
:103610002A5F3F4F9281891301C012823196E217CF
:10362000F307C1F7089581E090E0E0911101F09176
:103630001201E80FF91F1082019688309105A9F751
:1036400008958091F10208959091F102892B809361
:10365000F102089580959091F10289238093F102FF
:1036600008958093F10208951092F10208959091C7
:10367000F002892B8093F002089580959091F002DA
:1036800089238093F00208951092F00208958093A8
:10369000E70208951092E702089580911101909138
:1036A0001201FC0131969C01285F3F4F80E091910F
:1036B00091118F5FE217F307D1F70895E09111019F
:1036C000F09112018091F1028083E0911101F0915B
:1036D000120190818091F002892B80838091E70212
:1036E000882361F0E0911101F09112019081892B02
:1036F00080830E944D1B81111092E702809111017D
:10370000909112010C94BE0E909339018093380170
:1037100008958295982F9373292F220F220F982FA7
:103720009C7C96959695922B892F8575880F9A7A11
:103730009695892B08950895CF93DF9300D000D0FC
:103740001F92CDB7DEB70F900F900F900F900F9094
:10375000DF91CF910895089508950C94171008955E
:1037600080E0089580910703843021F11092F302E4
:1037700020E488E190E00FB6F894A895809360006B
:103780000FBE2093600083B7817F846083BF83B7BF
:10379000816083BF7894889583B78E7F83BF0FB68F
:1037A000F894A895809160008861809360001092E1
:1037B00060000FBE0895CF930E944F100E947206C2
:1037C0000E945010C0E08C2F0E940007811104C09D
:1037D000CF5FC830C1F701C081E0CF9108950E944A
:1037E00019100C94D4141F920F920FB60F9211243B
:1037F0008F939F93AF93BF938091F302811113C076
:103800008091F4029091F502A091F602B091F70236
:103810004196A11DB11D8093F4029093F502A093EF
:10382000F602B093F702BF91AF919F918F910F90E5
:103830000FBE0F901F90189582E084BD93E095BD58
:103840009AEF97BD80936E0008952FB7F8948091FA
:10385000F4029091F502A091F602B091F7022FBF09
:1038600008952FB7F8946091F4027091F502809159
:10387000F6029091F7022FBF0895CF92DF92EF9258
:10388000FF920F931F932FB7F8944091F402509139
:10389000F5026091F6027091F7022FBF6A017B0179
:1038A000EE24FF248C0120E030E0C016D106E206B1
:1038B000F30610F4415051099A01281B390BC90134
:1038C0001F910F91FF90EF90DF90CF9008951F927E
:1038D0000F920FB60F9211248F939F93AF93BF93C4
:1038E0008091F4029091F502A091F602B091F70256
:1038F0000196A11DB11D8093F4029093F502A0934F
:10390000F602B093F702BF91AF919F918F910F9004
:103910000FBE0F901F9018950E94010CF8942FEF86
:1039200087EA91E6215080409040E1F700C0000016
:1039300087E090EBDC018093110390931203A09336
:103940001303B09314039CE088E10FB6F894A89594
:10395000809360000FBE90936000FFCFE92FF0E0EE
:1039600093E0EE0FFF1F9A95E1F7E80FF11DEA547F
:10397000FF4F9491892F8F7092959F700895CF93E8
:10398000C82FCB010E94AE1C492F90E0242F30E0BD
:1039900054E0220F331F5A95E1F7282B392B20389A
:1039A000310519F480E090E017C0EC2FF0E023E03F
:1039B000EE0FFF1F2A95E1F74770E40FF11D34E089
:1039C000EE0FFF1F3A95E1F7E80FF91FEE0FFF1F0B
:1039D000E050F84985919491CF91089580E090E06E
:1039E00008950895CF92DF92EF92FF920F931F9365
:1039F000CF936C01C0E08C2F0E94000700E010E024
:103A0000E82EF12CC701002E02C0959587950A94E7
:103A1000E2F780FF15C0602F7C2F80E00E94BF1C62
:103A20008C159D0559F0292F207E392F307C11F0FF
:103A3000203A31F490E0C816D90611F481E009C0AB
:103A40000F5F1F4F08301105E9F6CF5FC83099F6B8
:103A500080E0CF911F910F91FF90EF90DF90CF907A
:103A60000895CF93DF93EC018CE290E00E94F21C6A
:103A7000882329F0CE01DF91CF910C94F21C80E0D5
:103A8000DF91CF910895CF930E94A41E811102C0AF
:103A90000E948A1E89E293E00E94A305C5E6C150F8
:103AA00049F00E9472068FE39CE90197F1F700C08C
:103AB0000000F5CF82E293E00E94A30589E290E046
:103AC0000E94311D811124C18AE290E00E94311DC3
:103AD00081110E948A1E85E090E00E94311D8111B3
:103AE0000E948C1C0E94AF1B0E94AF1E8093F202AA
:103AF00087E090E00E94311D8823C1F18BE190E0C6
:103B00000E94311D882351F08091F20281FB22270F
:103B100020F991E0922790FB81F90FC08EE090E0B0
:103B20000E94311D882361F08091F20282FB2227DE
:103B300020F991E0922790FB82F98093F20216C05F
:103B400080E190E00E94311D9091F202882341F0C3
:103B500093FB222720F981E0822780FB93F904C0A0
:103B6000892F809580FB90F99093F2028091F20268
:103B70000E94B31E0E94C11E8093100380EE90E04D
:103B80000E94311D882341F080911003982F909559
:103B900090FB80F98093100389E390E00E94311D2F
:103BA000882359F08091100381FB222720F991E0AE
:103BB000922790FB81F98093100382EE90E00E949F
:103BC000311D882359F08091100382FB222720F9B0
:103BD00091E0922790FB82F98093100386EE90E0AB
:103BE0000E94311D882359F08091100383FB222706
:103BF00020F991E0922790FB83F98093100383EEE4
:103C000090E00E94311D882359F08091100384FBBD
:103C1000222720F991E0922790FB84F980931003EA
:103C200085E390E00E94311D882359F080911003B4
:103C300085FB222720F991E0922790FB85F980935C
:103C4000100381E390E00E94311D882359F0809198
:103C5000100386FB222720F991E0922790FB86F93A
:103C60008093100381E190E00E94311D882359F078
:103C70008091100387FB222720F991E0922790FB87
:103C800087F980931003809110030E94C51E87E27C
:103C900090E00E94311DC82F8EE190E00E94311DFE
:103CA0008111C2608FE190E00E94311D8111C460DA
:103CB00080E290E00E94311D8111C86081E290E0B5
:103CC0000E94311D8111C06182E290E00E94311D8D
:103CD0008111C06283E290E00E94311D8111C064B5
:103CE00084E290E00E94311D882311F0C06802C078
:103CF000CC2329F08C2F0E94BC1E6C2F03C00E9485
:103D0000B81E682F70E080E090E0CF910C944B19C2
:103D1000CF9108956DEE7EEF80E090E00E94132831
:103D200060E082E090E00E94052860E083E090E09F
:103D30000E94052860E084E090E00E94052860E091
:103D400085E090E00C94052880E090E00E94FF2739
:103D500021E08D3E9E4F09F020E0822F089582E001
:103D600090E00C94F727682F82E090E00C940528EF
:103D700083E090E00C94F727682F83E090E00C94A8
:103D8000052884E090E00C94F727682F84E090E009
:103D90000C9405288091FA0280FF0CC080911601D6
:103DA00090E065E070E00E94B8279595879595951D
:103DB00087952EC081FF0AC08091160190E065E0D2
:103DC00070E00E94B8279595879522C082FF08C0B1
:103DD0008091160190E065E070E00E94B82718C05D
:103DE0002091FB022223D9F030911501231780F78F
:103DF0008091160190E065E070E00E94B827622F84
:103E000070E00E94B827632F70E00E94C927CB01A1
:103E10008038910538F4009739F481E005C085E0D9
:103E200090E008958FE7089508958091FA0280FF49
:103E300008C06091140170E0759567957595679558
:103E400023C081FF06C06091140170E075956795ED
:103E50001BC082FF04C06091140170E012C0609129
:103E6000FB026623A9F0209113016217A0F780914D
:103E7000140170E090E00E94B827622F70E00E9469
:103E8000C9276038710540F46115710519F406C041
:103E900061E070E0862F08958FE7089581E008952E
:103EA000803F21F40E94CA1E819504C0813F29F4FD
:103EB0000E94CA1E8093FE020895823F21F40E9450
:103EC000CA1E819504C0833F29F40E94CA1E8093B4
:103ED000FD020895893F19F40E94151F05C08A3F0D
:103EE00031F40E94151F81958093FF0208958B3F46
:103EF00021F40E94151F819504C08C3F29F40E9473
:103F0000151F809300030895843F21F48091FC02E3
:103F1000816017C0853F21F48091FC02826011C04E
:103F2000863F21F48091FC0284600BC0873F21F41E
:103F30008091FC02886005C0883F31F48091FC02CA
:103F400080618093FC0208958D3F21F48091FA02F4
:103F500081600BC08E3F21F48091FA02826005C01F
:103F60008F3F29F48091FA0284608093FA020895C9
:103F7000803F39F48091FE0287FF6CC01092FE02F0
:103F800069C0813F29F48091FE021816BCF362C01B
:103F90009091FD02823F29F497FF5CC01092FD02D0
:103FA00059C0833F19F41916CCF354C0893F41F42A
:103FB0008091FF0218160CF04DC01092FF024AC00B
:103FC0008A3F29F48091FF0287FF44C0F6CF8B3FE0
:103FD00039F48091000387FF3DC0109200033AC07E
:103FE0008C3F29F4809100031816BCF333C0843F42
:103FF00021F48091FC028E7F17C0853F21F48091CF
:10400000FC028D7F11C0863F21F48091FC028B7FE2
:104010000BC0873F21F48091FC02877F05C0883F59
:1040200031F48091FC028F7E8093FC0213C08D3F9F
:1040300021F48091FA028E7F0BC08E3F21F4809193
:10404000FA028D7F05C08F3F29F48091FA028B7FA1
:104050008093FA028091FD0281110EC08091FE02D0
:1040600081110AC08091FF02811106C08091000376
:10407000811102C01092FB0208958091F20283FF29
:104080007EC085E693E00E94A3058091FC021F920A
:104090008F9380E693E09F938F930E943C068EE57A
:1040A00093E00E94A3058091FD02282F082E000CAA
:1040B000330B3F938F938BE593E09F938F930E94F5
:1040C0003C0689E593E00E94A3058091FE02282F1B
:1040D000082E000C330B3F938F9386E593E09F935C
:1040E0008F930E943C0684E593E00E94A305809193
:1040F000FF02282F082E000C330B3F938F9381E58E
:1041000093E09F938F930E943C068FE493E00E947C
:10411000A30580910003282F082E000C330B3F933A
:104120008F938CE493E09F938F930E943C0689E4E5
:1041300093E00E94A3058091FB021F928F9386E477
:1041400093E09F938F930E943C0684E493E00E9447
:10415000A3058091FA021F928F9381E493E09F93CD
:104160008F930E943C068EE393E00E94A3058DB7D7
:104170009EB74C960FB6F8949EBF0FBE8DBF8CEFC6
:1041800092E00E94070F0E94251C9093F9028093F1
:10419000F80208951F93CF93DF938091F8029091D6
:1041A000F9020E943D1CFC012091FB02222321F018
:1041B0008091170190E007C08091180190E06AE0BB
:1041C00070E00E94B827E817F90708F485C08091CD
:1041D000FD02C091FE02D091FF02109100038111F7
:1041E00007C0C11175C0D11173C0111171C074C065
:1041F0002F3F19F02F5F2093FB02181624F40E9422
:10420000CA1E8093FD028091FD0287FF05C00E94B7
:10421000CA1E81958093FD021C1624F40E94CA1EBA
:104220008093FE028091FE0287FF05C00E94CA1E95
:1042300081958093FE026091FD02662331F1C09169
:10424000FE02CC2311F1062E000C770B880B990B84
:104250000E94B72623E333E343E35FE30E941B2777
:104260000E947F266093FD026C2FCC0F770B880B8A
:10427000990B0E94B72623E333E343E35FE30E94F5
:104280001B270E947F266093FE021D1624F40E94C5
:10429000151F8093FF028091FF0287FF05C00E94D7
:1042A000151F81958093FF02111624F40E94151F9B
:1042B000809300038091000387FF05C00E94151FB3
:1042C000819580930003DF91CF911F910C943D2045
:1042D0002F3F09F08FCFA0CFDF91CF911F9108958D
:1042E000ECEFF2E085E0DF011D928A95E9F710928C
:1042F000FB021092FA02089588E895E00E94A30557
:104300001F9281E08F931F9285E08F938AE395E05F
:104310009F938F930E943C060F900F900F900F90E9
:104320000F900F9008958330E9F128F4813061F007
:10433000823009F10895853009F462C008F449C05B
:10434000863009F474C0089580911801262F30E05A
:10435000280F311D2F3F310524F4680F6093180199
:1043600003C08FEF80931801809118011F928F93E3
:1043700083E794E072C080911701262F30E0280F68
:10438000311D2F3F310524F4680F6093170103C0DE
:104390008FEF80931701809117011F928F9381E611
:1043A00094E05BC080911601262F30E0280F311D6C
:1043B0002F3F310524F4680F6093160103C08FEF7F
:1043C00080931601809116011F928F938EE494E0E2
:1043D00044C080911501262F30E0280F311D2F3F5A
:1043E000310524F4680F6093150103C08FEF8093AB
:1043F0001501809115011F928F9389E394E02DC0E0
:1044000080911401262F30E0280F311D2F3F3105F8
:1044100024F4680F6093140103C08FEF809314019C
:10442000809114011F928F9380E294E016C08091D6
:104430001301262F30E0280F311D2F3F310524F4C2
:10444000680F6093130103C08FEF80931301809175
:1044500013011F928F9385E094E09F938F930E94A6
:104460003C060F900F900F900F900895833081F1CC
:1044700028F4813059F08230D1F00895853009F464
:1044800049C0B8F1863009F456C0089580911801EA
:10449000681720F4861B8093180102C0109218013F
:1044A000809118011F928F9386EF93E054C0809102
:1044B0001701681720F4861B8093170102C0109221
:1044C0001701809117011F928F9384EE93E043C0F0
:1044D00080911601681720F4861B8093160102C094
:1044E00010921601809116011F928F9381ED93E037
:1044F00032C080911501681720F4861B8093150146
:1045000002C010921501809115011F928F938CEBC0
:1045100093E021C080911401681720F4861B8093DA
:10452000140102C010921401809114011F928F9304
:1045300083EA93E010C080911301681720F4861B72
:104540008093130102C010921301809113011F92F6
:104550008F9388E893E09F938F930E943C060F907F
:104560000F900F900F900895CF93C82F1F928F93A5
:104570008DE896E09F938F930E943C0681E090E047
:10458000A0E0B0E0BC01CD0104C0660F771F881F1A
:10459000991FCA95D2F70E944B190F900F900F9058
:1045A0000F90CF910C94D414CF938732B0F58E3105
:1045B00008F040C28E3009F4BEC100F5873009F41E
:1045C0008DC1A8F4863009F039C28091F202817F52
:1045D0008E7F8093F20282E996E00E94A3058DE827
:1045E0009AE00E94A30581E08093020375C18830A0
:1045F00009F43FC08B3009F46BC120C2863109F445
:10460000E0C120F4803109F4AAC118C2893109F44B
:10461000C1C18B3109F47BC111C2883309F458C17F
:1046200050F4893209F404C2853309F401C2873297
:1046300009F004C2FDC1833409F4FAC128F48A33B5
:1046400008F4FCC18953F7C1883409F0F7C10E940E
:10465000D4148CE79AE00E94A3059FEF23ED80E33A
:10466000915020408040E1F700C000000E948C1C67
:1046700033C181E99AE00E94A30589E898E00E948D
:10468000A3050E94B81E1F928F9386E898E09F931F
:104690008F930E943C0684E898E00E94A3050E9444
:1046A000AF1EC82F81E798E00E94A3051F92CF9309
:1046B0008CE698E09F938F930E943C068AE698E0F0
:1046C0000E94A30580E698E00E94A3058C2F8170CC
:1046D0001F928F938DE598E09F938F930E943C06E5
:1046E0008BE598E00E94A30581E598E00E94A30570
:1046F000C1FB882780F91F928F938EE498E09F93E7
:104700008F930E943C068CE498E00E94A30580E40D
:1047100098E00E94A305C2FB882780F91F928F931F
:104720008DE398E09F938F930E943C068BE398E083
:104730000E94A30582E398E00E94A305C3FBCC2757
:10474000C0F91F92CF938FE298E09F938F930E94BE
:104750003C068DE298E00E94A3050E94C11EC82F6E
:1047600089E198E00E94A3051F92CF9384E198E02D
:104770009F938F930E943C0682E198E00E94A305DC
:1047800089EF97E00E94A3058C2F81701F928F9371
:1047900086EF97E09F938F930E943C068DB79EB75C
:1047A00080960FB6F8949EBF0FBE8DBF84EF97E042
:1047B0000E94A3058DED97E00E94A305C1FB882709
:1047C00080F91F928F938AED97E09F938F930E94B9
:1047D0003C0688ED97E00E94A30586EC97E00E94D6
:1047E000A305C2FB882780F91F928F9383EC97E083
:1047F0009F938F930E943C0681EC97E00E94A30553
:104800008FEA97E00E94A305C3FB882780F91F92D7
:104810008F938CEA97E09F938F930E943C068AEADD
:1048200097E00E94A30580EA97E00E94A305C4FBDD
:10483000882780F91F928F938DE997E09F938F933C
:104840000E943C068BE997E00E94A30589E897E067
:104850000E94A305C5FB882780F91F928F9386E8E5
:1048600097E09F938F930E943C0684E897E00E9414
:10487000A30588E697E00E94A305C6FB882780F978
:104880001F928F9385E697E09F938F930E943C063B
:1048900083E697E00E94A3058BE597E00E94A305BD
:1048A000C7FBCC27C0F91F92CF9388E597E09F9371
:1048B0008F930E943C0686E597E00E94A3058DB782
:1048C0009EB74C960FB6F8949EBF0FBE8DBF04C026
:1048D00089EB96E00E94A305C1E0B5C08091F20289
:1048E000C82FC17080FF09C08FE69AE00E94A3051F
:1048F0008091F202817F8E7F47C083E69AE00E941A
:10490000A3058091F20281608093F202E5CF90913D
:10491000F20291FBCC27C0F981E0C827892FC0FBA8
:1049200081F98093F202CC2319F086E59AE027C042
:1049300088E49AE0CFCF9091F20292FBCC27C0F9A5
:1049400081E0C827892FC0FB82F98093F202CC2333
:1049500019F089E39AE013C089E29AE0BBCF909105
:10496000F20293FBCC27C0F981E0C827892FC0FB56
:1049700083F98093F202CC2351F08DE19AE00E94FA
:10498000A3058091F20281608093F2025CC080E115
:104990009AE0A0CF81E09AE00E94A30589ED99E01A
:1049A0000E94A30587EA99E00E94A3058FE799E09A
:1049B0000E94A30580E399E00E94A30584E099E0AA
:1049C00089CF86EF98E00E94A3050E94B20E1F9245
:1049D0008F938CED98E09F938F930E943C0680917B
:1049E00010011F928F9385EC98E09F938F930E9404
:1049F0003C06809157021F928F9382EB98E09F9321
:104A00008F930E943C060E94311C9F938F937F934B
:104A10006F938BE998E09F938F930E943C068DB72C
:104A20009EB742960FB6F8949EBF0FBE8DBF54CF6F
:104A300080E001C08D510E94B4224ECF89E998E0F8
:104A40000E94A305C0E08C2FCF91089580E00895C7
:104A50000C942625CF93C82F80910203813071F0EA
:104A600020F0823009F44BC042C1E0911101F09175
:104A700012018081823209F03CC107C0E09111012E
:104A8000F09112018081823261F48C2F0E942825DE
:104A9000811104C08C2F0E94D4222FC081E090E0AD
:104AA0002CC08C2F0E942625811126C0C431E1F034
:104AB00070F4CB3081F0C031D1F40E947C2185E8C4
:104AC00096E00E94A30582E08093020315C0C932DC
:104AD00059F0C83361F482E996E00E94A30589E8A1
:104AE00096E00E94A30508C01092020304C183E867
:104AF00096E00E94A305FFC081E08170FEC0C43231
:104B000028F5CE3108F0C1C0CB30A1F1D0F4C730C8
:104B100009F0D3C08EE18093180182E380931701DE
:104B20008AE08093160184E18093150188E08093E8
:104B3000140188E28093130189E295E00E94A305A5
:104B4000BFC0C33149F1C431C1F0B7C0CB3409F49F
:104B5000A9C028F4C93289F0C83361F0AEC0C135AC
:104B600009F49EC0C23509F499C0CE3409F0A5C03D
:104B70006AE09EC00E947C21A3C08091010388232B
:104B800019F0109201039CC086E395E00E94A305F2
:104B900081E080930203B1C080E195E00E94A3050B
:104BA0008EEF94E00E94A305809118011F928F93CD
:104BB0008BEF94E09F938F930E943C0689EF94E0E3
:104BC0000E94A30587EE94E00E94A305809117013F
:104BD0001F928F9384EE94E09F938F930E943C06E4
:104BE00082EE94E00E94A30583ED94E00E94A30569
:104BF000809116011F928F9380ED94E09F938F9385
:104C00000E943C068EEC94E00E94A3058DEB94E09C
:104C10000E94A305809115011F928F938AEB94E067
:104C20009F938F930E943C0688EB94E00E94A3051B
:104C300083EA94E00E94A305809114011F928F9350
:104C400080EA94E09F938F930E943C068EE994E063
:104C50000E94A30587E894E00E94A30580911301B8
:104C60001F928F9384E894E09F938F930E943C0659
:104C700082E894E00E94A3058DB79EB748960FB6D0
:104C8000F8949EBF0FBE8DBF1BC0CE51EC2FF0E03D
:104C9000E25DFE4F80818093010312C061E003C09A
:104CA00061E006C06AE0809101030E94932108C080
:104CB000809101030E94362203C087E295E013C071
:104CC00080910103882369F01F928F9381E295E020
:104CD0009F938F930E943C060F900F900F900F9020
:104CE00004C08EE195E00E94A30581E006C0109209
:104CF000020380E002C080E000CFCF9108950E94BF
:104D000086266894B1110C94152708950E94FA26FE
:104D100088F09F5798F0B92F9927B751B0F0E1F07C
:104D2000660F771F881F991F1AF0BA95C9F714C02C
:104D3000B13091F00E941427B1E008950C9414272B
:104D4000672F782F8827B85F39F0B93FCCF3869565
:104D500077956795B395D9F73EF4909580957095C2
:104D600061957F4F8F4F9F4F0895E89409C097FB3F
:104D70003EF490958095709561957F4F8F4F9F4F32
:104D80009923A9F0F92F96E9BB279395F695879576
:104D900077956795B795F111F8CFFAF4BB0F11F439
:104DA00060FF1BC06F5F7F4F8F4F9F4F16C08823E0
:104DB00011F096E911C0772321F09EE8872F762F16
:104DC00005C0662371F096E8862F70E060E02AF057
:104DD0009A95660F771F881FDAF7880F9695879543
:104DE00097F9089557FD9058440F551F59F05F3FAC
:104DF00071F04795880F97FB991F61F09F3F79F0FD
:104E000087950895121613061406551FF2CF46957E
:104E1000F1DF08C0161617061806991FF1CF869500
:104E20007105610508940895E894BB2766277727E4
:104E3000CB0197F908950E942D270C94A7270E9473
:104E4000992738F00E94A02720F0952311F00C94A8
:104E500090270C9496270C9415270E94F22678F33D
:104E60009923C9F35523B9F3950F50E0551FAA278D
:104E7000EE27FF27BB2700240894679520F4E20F54
:104E8000F31FB41F0A1E220F331F441FAA1F66956B
:104E9000A9F7779530F4F30FB41F0A1E121E08F419
:104EA0006395330F441FAA1F221F769599F78795A4
:104EB00020F4B40F0A1E121E631F440FAA1F221FE4
:104EC000331F8695A9F7862F712D602D11249F57CA
:104ED00050409AF0F1F088234AF0EE0FFF1FBB1FFD
:104EE000661F771F881F91505040A9F79E3F5105BC
:104EF00080F00C9490270C9415275F3FE4F3983EC4
:104F0000D4F3869577956795B795F795E7959F5F65
:104F1000C1F7FE2B880F911D9695879597F90895F7
:104F200097F99F6780E870E060E008959FEF80EC5C
:104F3000089500240A9416161706180609060895FF
:104F400000240A9412161306140605060895092E65
:104F50000394000C11F4882352F0BB0F40F4BF2BD4
:104F600011F460FF04C06F5F7F4F8F4F9F4F089514
:104F70000024552704C0080E591F880F991F009759
:104F800029F076956795B8F37105B9F7802D952FBF
:104F9000089597FB072E16F4009407D077FD09D0EB
:104FA0000E94E32707FC05D03EF4909581959F4F22
:104FB0000895709561957F4F0895EE0FFF1F05903E
:104FC000F491E02D0994AA1BBB1B51E107C0AA1F55
:104FD000BB1FA617B70710F0A61BB70B881F991F9A
:104FE0005A95A9F780959095BC01CD010895F9993E
:104FF000FECF92BD81BDF89A992780B50895A8E1AA
:10500000B0E042E050E00C941A28262FF999FECF28
:105010001FBA92BD81BD20BD0FB6F894FA9AF99AD5
:105020000FBE019608950E940528272F0C9406288C
:10503000DC01CB01FC01F999FECF06C0F2BDE1BD58
:10504000F89A319600B40D9241505040B8F7089547
:04505000F894FFCF02
:10505400054E010000FF0E079E077B074507110759
:1050640001E8022808140A321E404D36228A023D05
:10507400020702E50171018A01A301BC01000102DA
:085084000304050607080900FA
:106800000000000000000000040005000600070072
:10681000080009000A000B000C000D000E000F001C
:1068200010001100120013001400150016001700CC
:10683000180019001A001B001C001D001E001F007C
:10684000200021002200230024002500260027002C
:10685000280029002A002B002C002D002E002F00DC
:1068600030003100000033003400350036003700BE
:1068700038003900000000000000000000000000A7
:106880000000000000000000000000000000000008
:1068900000000000000000000000000000000000F8
:1068A00000000000000000000000000000000000E8
:1068B00000000000000000000000000000000000D8
:1068C00000000000000000006400E700000000007D
:1068D00000000000000000000000000000000000B8
:1068E0000000000000000000320000000000000076
:1068F000E000E100E300E200E400E500E6006500FE
:00000001FF
